:020000040000FA
:100000008501003065008601FF3066000515AF01EF
:10001000AD01C101C3013C30C20006088500372094
:100020000D2843084005031D26280608430503192B
:1000300008009030AD00442042084107AD00442044
:100040007F30AD0044204308C00408000608430583
:10005000031D08008030AD00442042084107AD0078
:1000600044200030AD0044204308C00608000130A1
:10007000AC00FF30AB000A30AA00AA0B3D28AB0B46
:100080003B28AC0B3928080005111830AF00AF0B26
:1000900047280830AB00AD0C0318512800000511AB
:1000A00054280515000000001730AF00AF0B56288C
:1000B000AB0B4B28000000000000000000000515FD
:0A00C0001A30AF00AF0B62280800F1
:02400E00F23F7F
:00000001FF
